:100000000C9438000C9455000C9455000C94550039
:100010000C9455000C9455000C9455000C9455000C
:100020000C9455000C9455000C9455000C945500FC
:100030000C9455000C9455000C9455000C945500EC
:100040000C9455000C94B2020C9455000C9455007D
:100050000C94DD0E0C9455000C9455000C94550036
:100060000C9455000C9455000C9455000C945500BC
:1000700011241FBECFEFD4E0DEBFCDBF13E0A0E060
:10008000B1E0E4E6F2E202C005900D92AE33B107B2
:10009000D9F714E0AEE3B3E001C01D92AB32B10773
:1000A000E1F70E9474000C9430110C940000DF936F
:1000B000CF93CDB7DEB7E4E3F0E08FEF8083EAE3E0
:1000C000F0E08EE28083ABE3B0E0EBE3F0E0808130
:1000D00082608C93ABE3B0E0EBE3F0E08081806280
:1000E0008C93CF91DF910895DF93CF93CDB7DEB797
:1000F0000E9457000E94A3020E94F70D7894A5E386
:10010000B0E0E5E3F0E0808181608C930E947602AC
:100110000E94EE020E9439030E9484030E94CF03D2
:100120000E941A040E9465040E94B0040E94FB040D
:100130000E94770680914003813031F41092400391
:100140000E9484100E94931080914D038130E1F44D
:10015000A5E3B0E0E5E3F0E0808184608C930E9449
:10016000F80C0E946D0F0E9404070E9419080E945B
:1001700049090E94BE050E949C06A5E3B0E0E5E3A4
:10018000F0E080818B7F8C9380913E03813091F6EB
:1001900010923E030E944605CDCFDF93CF93CDB79B
:1001A000DEB784E064E00E94EA0080E06CE40E9434
:1001B000EA0010924003809140038823E1F38CE62B
:1001C0006AE00E94EA0085E060E00E94EA00CF91C8
:1001D000DF910895DF93CF9300D000D0CDB7DEB785
:1001E0008B836C83ABE3B0E0EBE3F0E080818D7F49
:1001F0008C9387E08A8340C0ABE3B0E0EBE3F0E0B0
:100200008081877F8C9300000000000000008A81BD
:10021000282F332727FD309581E090E0022E02C081
:10022000880F991F0A94E2F7982F8B81892389837D
:100230008981882341F0ABE3B0E0EBE3F0E080811B
:1002400084608C9307C0ABE3B0E0EBE3F0E0808127
:100250008B7F8C930000000000000000ABE3B0E057
:10026000EBE3F0E0808188608C93000000000000E8
:1002700000008A8181508A838A8188230CF0BCCF58
:1002800087E08A8340C0ABE3B0E0EBE3F0E080813D
:10029000877F8C9300000000000000008A81282FD7
:1002A000332727FD309581E090E0022E02C0880FB1
:1002B000991F0A94E2F7982F8C8189238983898179
:1002C000882341F0ABE3B0E0EBE3F0E080818460B1
:1002D0008C9307C0ABE3B0E0EBE3F0E080818B7F71
:1002E0008C930000000000000000ABE3B0E0EBE303
:1002F000F0E0808188608C93000000000000000026
:100300008A8181508A838A8188230CF0BCCFABE339
:10031000B0E0EBE3F0E08081877F8C93ABE3B0E06B
:10032000EBE3F0E080818B7F8C93ABE3B0E0EBE319
:10033000F0E0808182608C930F900F900F900F906F
:10034000CF91DF910895DF93CF9300D000D0CDB748
:10035000DEB78C83ABE3B0E0EBE3F0E080818D7F30
:100360008C9387E08A834CC0ABE3B0E0EBE3F0E032
:100370008081877F8C930000000000000000000057
:100380000000000000008A81282F332727FD3095C8
:1003900081E090E0022E02C0880F991F0A94E2F7D4
:1003A000982F8C8189238B838B81181644F4ABE3BF
:1003B000B0E0EBE3F0E0808184608C9307C0ABE3B6
:1003C000B0E0EBE3F0E080818B7F8C9300000000D5
:1003D000000000000000000000000000ABE3B0E0FF
:1003E000EBE3F0E0808188608C9300000000000067
:1003F000000000000000000000008A8181508A8314
:100400008A8188230CF0B0CF1B82ABE3B0E0EBE332
:10041000F0E08081877F8C930000000000000000E6
:10042000000000000000000087E08A833EC0ABE3CC
:10043000B0E0EBE3F0E0808188608C93E9E3F0E0EA
:10044000808189838981882F90E08071907018164F
:1004500019068CF48A81282F332727FD309581E0F7
:1004600090E0022E02C0880F991F0A94E2F7982F9D
:100470008B81892B8B8300000000000000000000AE
:10048000000000000000ABE3B0E0EBE3F0E08081AF
:10049000877F8C9300000000000000000000000037
:1004A000000000008A8181508A838A8188230CF0B1
:1004B000BECFABE3B0E0EBE3F0E08081877F8C93CD
:1004C000ABE3B0E0EBE3F0E080818B7F8C93ABE3B8
:1004D000B0E0EBE3F0E0808182608C938B810F9041
:1004E0000F900F900F90CF91DF910895DF93CF93EE
:1004F000CDB7DEB70E94CD0010923E0380913E033F
:100500008823E1F30E9483050E941D0B10923E0395
:1005100080913E038823E1F310923E0380913E03D5
:100520008823E1F310923E0384E064E00E94EA0035
:1005300080E06CE40E94EA000E9446050E94DD050E
:10054000CF91DF910895DF93CF93CDB7DEB7E3E589
:10055000F0E082E08083E9E5F0E082E08083CF9103
:10056000DF9108951F920F920FB60F9211248F936F
:10057000DF93CF93CDB7DEB7809142038F5F809337
:10058000420380914203883409F581E0809341035E
:10059000109242038091E6038F5F8093E60380917F
:1005A000E603843629F41092E60381E080933E034B
:1005B0008091E5038F5F8093E5038091E5038A30A6
:1005C00029F41092E50381E080934003CF91DF91FD
:1005D0008F910F900FBE0F901F901895DF93CF93C0
:1005E000CDB7DEB780E062E40E94EA0010923E03DD
:1005F00080913E038823E1F310923E0389E060EC92
:100600000E94EA0010924003809140038823E1F3A6
:10061000109240031092E70317C09091E7038AE01D
:10062000692F0E94EA008091E703882F90E0FC0187
:10063000E95CFE4F90818BE0692F0E94EA00809177
:10064000E7038F5F8093E7038091E703863328F306
:1006500088E060EA0E94EA00109240038091400323
:100660008823E1F380E06CE40E94EA00CF91DF91FF
:100670000895DF93CF93CDB7DEB780E062E40E94A8
:10068000EA0010923E0380913E038823E1F310922A
:100690003E0389E061EC0E94EA00109240038091E1
:1006A00040038823E1F3109240031092E70317C040
:1006B0009091E7038AE0692F0E94EA008091E703A6
:1006C000882F90E0FC01E958FE4F90818BE0692F64
:1006D0000E94EA008091E7038F5F8093E703809197
:1006E000E703863328F388E060EA0E94EA0010926C
:1006F0004003809140038823E1F380E06CE40E9492
:10070000EA00CF91DF910895DF93CF93CDB7DEB7A5
:1007100080E062E40E94EA0010923E0380913E0372
:100720008823E1F310923E0389E062EC0E94EA0024
:1007300010924003809140038823E1F3109240031C
:100740001092E70317C09091E7038AE0692F0E9497
:10075000EA008091E703882F90E0FC01E954FE4F06
:1007600090818BE0692F0E94EA008091E7038F5F00
:100770008093E7038091E703863328F388E060EAFB
:100780000E94EA0010924003809140038823E1F325
:1007900080E06CE40E94EA00CF91DF910895DF933E
:1007A000CF93CDB7DEB780E062E40E94EA001092FA
:1007B0003E0380913E038823E1F310923E0389E0DB
:1007C00063EC0E94EA00109240038091400388236A
:1007D000E1F3109240031092E70317C09091E703F2
:1007E0008AE0692F0E94EA008091E703882F90E059
:1007F000FC01E950FE4F90818BE0692F0E94EA00D6
:100800008091E7038F5F8093E7038091E70386334E
:1008100028F388E060EA0E94EA0010924003809189
:1008200040038823E1F380E06CE40E94EA00CF916A
:10083000DF910895DF93CF93CDB7DEB780E062E418
:100840000E94EA0010923E0380913E038823E1F368
:1008500010923E0389E064EC0E94EA00109240038B
:10086000809140038823E1F3109240031092E70344
:1008700017C09091E7038AE0692F0E94EA008091F7
:10088000E703882F90E0FC01E95CFD4F90818BE04D
:10089000692F0E94EA008091E7038F5F8093E7034E
:1008A0008091E703863328F388E060EA0E94EA003B
:1008B00010924003809140038823E1F380E06CE4D0
:1008C0000E94EA00CF91DF910895DF93CF93CDB7D7
:1008D000DEB780E062E40E94EA0010923E0380915D
:1008E0003E038823E1F310923E0389E065EC0E9409
:1008F000EA0010924003809140038823E1F31092B4
:1009000040031092E70317C09091E7038AE0692F34
:100910000E94EA008091E703882F90E0FC01E958EB
:10092000FD4F90818BE0692F0E94EA008091E703E0
:100930008F5F8093E7038091E703863328F388E095
:1009400060EA0E94EA0010924003809140038823ED
:10095000E1F380E06CE40E94EA00CF91DF9108951A
:10096000DF93CF93CDB7DEB780E062E40E94EA0068
:1009700010923E0380913E038823E1F310923E03E0
:1009800089E066EC0E94EA001092400380914003E7
:100990008823E1F3109240031092E70317C090916F
:1009A000E7038AE0692F0E94EA008091E703882F1D
:1009B00090E0FC01E954FD4F90818BE0692F0E948B
:1009C000EA008091E7038F5F8093E7038091E7035C
:1009D000863328F388E060EA0E94EA001092400320
:1009E000809140038823E1F380E06CE40E94EA00F8
:1009F000CF91DF910895DF93CF93CDB7DEB780E03D
:100A000062E40E94EA0010923E0380913E03882334
:100A1000E1F310923E0389E067EC0E94EA00109235
:100A20004003809140038823E1F310924003109229
:100A3000E70317C09091E7038AE0692F0E94EA005C
:100A40008091E703882F90E0FC01E950FD4F9081F1
:100A50008BE0692F0E94EA008091E7038F5F80930B
:100A6000E7038091E703863328F388E060EA0E9479
:100A7000EA0010924003809140038823E1F380E074
:100A80006CE40E94EA00CF91DF910895DF93CF9349
:100A9000CDB7DEB789ED8093E70313C085E060E052
:100AA0000E94EA009091E70386E0692F0E94EA0025
:100AB00087E064E50E94EA008091E7038F5F8093FE
:100AC000E7038091E7038C3D48F385EE8093E703CD
:100AD00013C085E060E00E94EA009091E70386E0A1
:100AE000692F0E94EA0087E064E50E94EA00809195
:100AF000E7038F5F8093E7038091E703883E48F325
:100B0000CF91DF910895DF93CF93CDB7DEB7649790
:100B10000FB6F894DEBF0FBECDBF8DE589838EE59D
:100B20008A838FE58B8389E48C838BE58D838DE1CC
:100B30008E838CE58F83188680E2898789E28A8795
:100B400086E38B8781E48C878AE08D8781E48E87BA
:100B500081E08F8786E2888B87E062E09E012F5FCD
:100B60003F4FA90120E10E94080664960FB6F89451
:100B7000DEBF0FBECDBFCF91DF910895DF93CF933E
:100B8000CDB7DEB785E060E00E94EA0086E06FEC5A
:100B90000E94EA0087E06CE80E94EA0085E061E0DC
:100BA0000E94EA0086E06BE00E94EA0087E06DE8C0
:100BB0000E94EA00CF91DF910895DF93CF93CDB7E4
:100BC000DEB785E060E00E94EA0086E060E20E9415
:100BD000EA0087E060E80E94EA0085E060E00E94A9
:100BE000EA0086E06EE30E94EA0087E064E80E9483
:100BF000EA0085E060E00E94EA0086E06CE50E9481
:100C0000EA0087E068E80E94EA00CF91DF9108954A
:100C1000DF93CF93CDB7DEB72D970FB6F894DEBF35
:100C20000FBECDBF89876A875C874B872D878A85F2
:100C3000282F30E0C901880F991F820F931F9C0154
:100C4000220F331F220F331F820F931F880F991F0C
:100C50009C018985882F90E0820F931F98878F834E
:100C60008D85282F30E08F819885820F931F9E837A
:100C70008D831092E7038F8198859C838B8327C097
:100C80008B818A838B819C81892F9927898385E039
:100C900069810E94EA0086E06A810E94EA00409130
:100CA000E703242F30E08B859C85FC01E20FF31FC6
:100CB0008081982F842F8F5F8093E70387E0692FCF
:100CC0000E94EA008B819C8101969C838B832B81FF
:100CD0003C818D819E812817390790F22D960FB6A1
:100CE000F894DEBF0FBECDBFCF91DF910895DF93A3
:100CF000CF93CDB7DEB721E031E083E06EE0A9010C
:100D000029E00E940806CF91DF910895DF93CF93E9
:100D100000D0CDB7DEB78A838A81882321F48A8107
:100D20008652898303C08A818053898389810F9089
:100D30000F90CF91DF9108950F931F93DF93CF937F
:100D4000CDB7DEB72D970FB6F894DEBF0FBECDBF7F
:100D50008091F4039091F5032EE130E0B9010E94F7
:100D60000911CB019B838A838A819B819E012C5F21
:100D70003F4FB9014AE050E00E94D810CE010496DE
:100D80000E94BF1089831092E7031CC08091E70383
:100D9000082F10E08091E703282F30E0CE01049661
:100DA000FC01E20FF31F80810E948606282FCE01EE
:100DB0000996FC01E00FF11F20838091E7038F5F0C
:100DC0008093E7038091E703282F30E089819927FA
:100DD00087FD909528173907CCF299818BE0891B04
:100DE00099819E01275F3F4F6EE0A901292F0E9444
:100DF00008062D960FB6F894DEBF0FBECDBFCF917B
:100E0000DF911F910F910895DF93CF93CDB7DEB798
:100E100029970FB6F894DEBF0FBECDBF8091FC03BB
:100E20009091FD038E5590409C838B838B819C8198
:100E300023E030E0B9010E940911CB019A83898334
:100E400089819A818A30910524F089E090E09A8323
:100E5000898389819A81992314F41A8219822091B5
:100E600046033091470389819A818217930709F4D9
:100E7000D7C089819A81823091052CF484E060E1A9
:100E80000E94EA0004C084E060E00E94EA008981D8
:100E90009A81909347038093460380E88D8384E88A
:100EA0008E8388E88F8389819A819987888788854E
:100EB00099858430910509F45FC0888599858530CE
:100EC0009105DCF4888599858130910509F43FC04E
:100ED00088859985823091052CF4888599850097BD
:100EE00079F173C08885998582309105B9F188853B
:100EF000998583309105C9F168C0888599858730C7
:100F0000910509F44EC088859985883091055CF477
:100F10008885998585309105B1F1888599858630D8
:100F20009105C1F152C0888599858830910509F4F1
:100F30003FC0888599858930910509F440C045C036
:100F400080E88D8384E88E8388E88F833EC081E8C3
:100F50008D8384E88E8388E88F8337C082E88D8311
:100F600084E88E8388E88F8330C083E88D8384E8AB
:100F70008E8388E88F8329C083E88D8385E88E83FC
:100F800088E88F8322C083E88D8386E88E8388E893
:100F90008F831BC083E88D8387E88E8388E88F83E7
:100FA00014C083E88D8387E88E8389E88F830DC022
:100FB00083E88D8387E88E838AE88F8306C083E881
:100FC0008D8387E88E838BE88F8385E060E00E94C5
:100FD000EA0086E060E20E94EA009D8187E0692FD6
:100FE0000E94EA0085E060E00E94EA0086E06EE38D
:100FF0000E94EA009E8187E0692F0E94EA0085E056
:1010000060E00E94EA0086E06CE50E94EA009F81B1
:1010100087E0692F0E94EA0084E060E00E94EA0015
:1010200029960FB6F894DEBF0FBECDBFCF91DF91EA
:101030000895DF93CF9300D000D000D0CDB7DEB7B6
:101040008091EC039091ED0326E130E0B9010E941C
:101050000911CB0106969E838D838D819E819923F4
:101060000CF446C08D819E812AE030E0B9010E94D7
:101070000911CB018A838D819E812AE030E0B9017C
:101080000E9409118983898186958C5F89838A8171
:10109000282F30E086E890E0821B930B9C838B83A3
:1010A00020910D0130910E018B819C818217930755
:1010B00061F080910D0190910E010E94D0088B810A
:1010C0009C8169810E9407090AC090914B03898124
:1010D000981729F08B819C8169810E940709898179
:1010E00080934B038B819C8190930E0180930D0123
:1010F0008D819E8199230CF04AC08D819E819095AF
:1011000081959F4F9E838D838D819E812AE030E063
:10111000B9010E940911CB018A838D819E812AE049
:1011200030E0B9010E9409118983898186958983FC
:101130008A81882F90E08A579F4F9C838B832091D0
:101140000D0130910E018B819C818217930761F014
:1011500080910D0190910E010E94D0088B819C819D
:1011600069810E9407090AC090914B0389819817F1
:1011700029F08B819C8169810E9407098981809374
:101180004B038B819C8190930E0180930D012696D9
:101190000FB6F894DEBF0FBECDBFCF91DF9108959B
:1011A000DF93CF9300D000D000D0CDB7DEB79E83C1
:1011B0008D831C821B821DC08D818A838D819E81BF
:1011C000892F9927898385E069810E94EA0086E05A
:1011D0006A810E94EA0087E060E00E94EA008D8157
:1011E0009E814E969E838D838B819C8101969C83EC
:1011F0008B838B819C8188309105F0F226960FB607
:10120000F894DEBF0FBECDBFCF91DF910895DF937D
:10121000CF93CDB7DEB727970FB6F894DEBF0FBEDA
:10122000CDBF9E838D836F831C821B8224C08D81E2
:101230008A838D819E81892F9927898385E06981A1
:101240000E94EA0086E06A810E94EA008F81882F6E
:1012500090E0FC01E35DFE4F908187E0692F0E94E2
:10126000EA008D819E814E969E838D838B819C8129
:1012700001969C838B838B819C8188309105B8F289
:1012800027960FB6F894DEBF0FBECDBFCF91DF918A
:101290000895DF93CF9300D000D000D0CDB7DEB754
:1012A0008091EA039091EB0326E130E0B9010E94BE
:1012B0000911CB019E838D838D819E8199230CF42E
:1012C00056C08D819E812AE030E0B9010E9409114B
:1012D000CB018A838D819E812AE030E0B9010E9492
:1012E000091189838981869589838A81282F30E035
:1012F00087E090E0AC01421B530B9A01C901880FB3
:10130000991F820F931F9C01220F331F220F331F3F
:10131000820F931F880F991F0A969C838B832091BD
:101320000B0130910C018B819C818217930761F036
:1013300080910B0190910C010E941E0A8B819C816F
:1013400069810E947E0A0AC090914A038981981798
:1013500029F08B819C8169810E947E0A898180931A
:101360004A038B819C8190930C0180930B018D81AA
:101370009E8199230CF059C08D819E819095819515
:101380009F4F9E838D838D819E812AE030E0B9013D
:101390000E940911CB018A838D819E812AE030E071
:1013A000B9010E9409118983898186958C5F89839F
:1013B0008A81282F30E0C901880F991F820F931F5F
:1013C0009C01220F331F220F331F820F931F880FA0
:1013D000991F86509F4F9C838B8320910B013091E6
:1013E0000C018B819C818217930761F080910B0126
:1013F00090910C010E941E0A8B819C8169810E9440
:101400007E0A0AC090914A038981981729F08B813E
:101410009C8169810E947E0A898180934A038B8125
:101420009C8190930C0180930B0126960FB6F89443
:10143000DEBF0FBECDBFCF91DF910895DF93CF9375
:1014400000D000D000D0CDB7DEB79E838D838D81D4
:101450009E819C838B8318C08B818A838B819C8126
:10146000892F9927898385E069810E94EA0086E0B7
:101470006A810E94EA0087E060E00E94EA008B81B6
:101480009C8101969C838B838D819E819C01275F2B
:101490003F4F8B819C8182179307F0F280914A0322
:1014A000282F30E0C901880F991F820F931FFC017C
:1014B000EF5EFE4F80818823C1F08D819E818296F0
:1014C0009C838B838B818A838B819C81892F992735
:1014D000898385E069810E94EA0086E06A810E9432
:1014E000EA0087E060E00E94EA0026960FB6F894D2
:1014F000DEBF0FBECDBFCF91DF910895DF93CF93B5
:10150000CDB7DEB727970FB6F894DEBF0FBECDBFBD
:101510009E838D836F838D819E819C838B8324C06A
:101520008B8189838B819C81892F99278A8385E090
:101530006A810E94EA0086E069810E94EA008F8148
:10154000282F30E0C901880F991F820F931FFC01DB
:10155000E15FFE4F908187E0692F0E94EA008B8156
:101560009C8101969C838B838D819E819C01275F4A
:101570003F4F8B819C818217930790F28D819E81D2
:1015800004969C838B838B8189838B819C81892F9B
:1015900099278A8385E06A810E94EA0086E0698152
:1015A0000E94EA008F81282F30E0C901880F991F1F
:1015B000820F931FFC01E05FFE4F908187E0692F4F
:1015C0000E94EA008F81282F30E0C901880F991FFF
:1015D000820F931FFC01EF5EFE4F8081882321F173
:1015E0008D819E8182969C838B838B8189838B8165
:1015F0009C81892F99278A8385E06A810E94EA006D
:1016000086E069810E94EA008F81282F30E0C901BD
:10161000880F991F820F931FFC01EF5EFE4F908190
:1016200087E0692F0E94EA0027960FB6F894DEBF84
:101630000FBECDBFCF91DF910895DF93CF93CDB78C
:10164000DEB785E060E00E94EA0086E063E80E9481
:10165000EA0087E060E90E94EA0085E060E00E941D
:10166000EA0086E064E80E94EA0087E061E90E94FF
:10167000EA0085E060E00E94EA0086E065E80E94FA
:10168000EA0087E062E90E94EA0085E060E00E94EB
:10169000EA0086E066E80E94EA0087E063E90E94CB
:1016A000EA0085E060E00E94EA0086E067E80E94C8
:1016B000EA0087E064E90E94EA0085E060E00E94B9
:1016C000EA0086E068E80E94EA0087E065E90E9497
:1016D000EA0085E060E00E94EA0086E069E80E9496
:1016E000EA0087E066E90E94EA0085E060E00E9487
:1016F000EA0086E06AE80E94EA0087E067E90E9463
:10170000EA0085E060E00E94EA0086E061EA0E946B
:10171000EA0087E068E90E94EA0085E060E00E9454
:10172000EA0086E062EA0E94EA0087E069E90E9436
:10173000EA0085E060E00E94EA0086E063EA0E9439
:10174000EA0087E06AE90E94EA0085E060E00E9422
:10175000EA0086E064EA0E94EA0087E06BE90E9402
:10176000EA0085E060E00E94EA0086E065EA0E9407
:10177000EA0087E06CE90E94EA0085E060E00E94F0
:10178000EA0086E066EA0E94EA0087E06DE90E94CE
:10179000EA0085E060E00E94EA0086E067EA0E94D5
:1017A000EA0087E06EE90E94EA0085E060E00E94BE
:1017B000EA0086E068EA0E94EA0087E06FE90E949A
:1017C000EA0085E060E00E94EA0086E06FEB0E949C
:1017D000EA0087E060EA0E94EA0085E060E00E949B
:1017E000EA0086E060EC0E94EA0087E061EA0E947D
:1017F000EA0085E060E00E94EA0086E061EC0E9479
:10180000EA0087E062EA0E94EA0085E060E00E9468
:10181000EA0086E062EC0E94EA0087E063EA0E9448
:10182000EA0085E060E00E94EA0086E063EC0E9446
:10183000EA0087E064EA0E94EA0085E060E00E9436
:10184000EA0086E064EC0E94EA0087E065EA0E9414
:10185000EA0085E060E00E94EA0086E065EC0E9414
:10186000EA0087E066EA0E94EA0085E060E00E9404
:10187000EA0086E066EC0E94EA0087E067EA0E94E0
:10188000EA0085E060E00E94EA0086E06DED0E94DB
:10189000EA0087E068EA0E94EA0085E060E00E94D2
:1018A000EA0086E06EED0E94EA0087E069EA0E94A5
:1018B000EA0085E060E00E94EA0086E06FED0E94A9
:1018C000EA0087E06AEA0E94EA0085E060E00E94A0
:1018D000EA0086E060EE0E94EA0087E06BEA0E9480
:1018E000EA0085E060E00E94EA0086E061EE0E9486
:1018F000EA0087E06CEA0E94EA0085E060E00E946E
:10190000EA0086E062EE0E94EA0087E06DEA0E944B
:10191000EA0085E060E00E94EA0086E063EE0E9453
:10192000EA0087E06EEA0E94EA0085E060E00E943B
:10193000EA0086E064EE0E94EA0087E06FEA0E9417
:10194000EA0085E060E00E94EA0086E06BEF0E941A
:10195000EA0087E060EB0E94EA0085E060E00E9418
:10196000EA0086E06CEF0E94EA0087E061EB0E94EB
:10197000EA0085E060E00E94EA0086E06DEF0E94E8
:10198000EA0087E062EB0E94EA0085E060E00E94E6
:10199000EA0086E06EEF0E94EA0087E063EB0E94B7
:1019A000EA0085E060E00E94EA0086E06FEF0E94B6
:1019B000EA0087E064EB0E94EA0085E061E00E94B3
:1019C000EA0086E060E00E94EA0087E065EB0E94A2
:1019D000EA0085E061E00E94EA0086E061E00E94A2
:1019E000EA0087E066EB0E94EA00CF91DF9108955C
:1019F000DF93CF93CDB7DEB767970FB6F894DEBF0E
:101A00000FBECDBF83E090E09C8B8B8B1A82198236
:101A100083E990E09C838B8310924D03DAC08B891D
:101A20009C89FC01E25BFC4F8081882F90E0CD9780
:101A30009A8B898B8B899C8901969C8B8B8B8B894C
:101A40009C89FC01E25BFC4F8081882F90E0CD9760
:101A5000988B8F878B899C8901969C8B8B8B8B892C
:101A60009C89FC01E25BFC4F8081882F90E0CD9740
:101A70009E878D878B899C8901969C8B8B8B8B890C
:101A80009C89FC01E25BFC4F8081882F90E0CD9720
:101A90009C878B878B899C8901969C8B8B8B8989F2
:101AA0009A899C01220F331F220F331F8F8598893B
:101AB000959587959595879595958795959587950E
:101AC000822B932B9A8789878F8598898295929507
:101AD000907F9827807F98279C0130708D859E8508
:101AE0009595879595958795822B932B98878F83CE
:101AF0008D859E8500249695879507949695879564
:101B00000794982F802D9C0130708B859C85822BAB
:101B1000932B9E838D831F8A8B819C81009711F06C
:101B200081E08F8B8B819C8101979C838B838F8934
:101B3000882309F453C020913703309138038981F9
:101B40009A81F901E80FF91F8985808389819A813B
:101B500001969A8389831E8A8B819C81009711F05C
:101B600081E08E8B8B819C8101979C838B838E89F6
:101B70008823A1F1209137033091380389819A811C
:101B8000F901E80FF91F8F81808389819A8101967D
:101B90009A8389831D8A8B819C81009711F081E053
:101BA0008D8B8B819C8101979C838B838D8988236E
:101BB000A9F0209137033091380389819A81F90186
:101BC000E80FF91F8D81808389819A8101969A831C
:101BD00089838B819C81009709F021CF67960FB68E
:101BE000F894DEBF0FBECDBFCF91DF910895DF9394
:101BF000CF93CDB7DEB7E9E2F0E082E28083E0E4A4
:101C0000F0E01082E0E2F0E082E28083ECE5F0E0D8
:101C10001082A2E3B0E0E2E3F0E0808181608C9387
:101C2000A8E3B0E0E8E3F0E0808184608C93EAE22E
:101C3000F0E088E98083E0E4F0E086E88083EBE28E
:101C4000F0E082EC8083E1E2F0E088E98083ECE57B
:101C5000F0E086E88083E2E2F0E082EC8083CF91DE
:101C6000DF910895DF93CF930F92CDB7DEB78983CD
:101C7000EBE2F0E08081882F90E080729070009716
:101C8000B9F3ECE2F0E0898180830F90CF91DF918E
:101C90000895DF93CF9300D000D000D0CDB7DEB74A
:101CA0009E838D838D819E810E94BF109C838B8338
:101CB0001A8219820FC02D813E8189819A81F90192
:101CC000E80FF91F80810E94320E89819A81019666
:101CD0009A83898329813A818B819C81821793071A
:101CE00050F7809139030E94320E80913A030E948E
:101CF000320E26960FB6F894DEBF0FBECDBFCF9141
:101D0000DF910895DF93CF93CDB7DEB766970FB617
:101D1000F894DEBF0FBECDBF9E8B8D8B8D899E89C3
:101D20009E012F5F3F4FB9014AE050E00E94D8105A
:101D3000CE0101960E94490E66960FB6F894DEBF5A
:101D40000FBECDBFCF91DF910895DF93CF9300D029
:101D5000CDB7DEB78A8387E089831FC08A81482F89
:101D600050E08981282F332727FD309581E090E0CE
:101D7000022E02C0880F991F0A94E2F7842395234C
:101D80001816190624F481E30E94320E03C080E382
:101D90000E94320E89818150898389818823F4F6DB
:101DA000809139030E94320E80913A030E94320ED4
:101DB0000F900F90CF91DF9108951F920F920FB661
:101DC0000F9211242F933F938F939F93AF93BF93C1
:101DD000EF93FF93DF93CF9300D0CDB7DEB7E3E26D
:101DE000F0E0808180932A0480912A048D30D9F418
:101DF00080914C038130B9F4A5E3B0E0E5E3F0E075
:101E00008081877F8C9310924C0381E080934D03F7
:101E10008091E403882F90E020912A04FC01E25B8A
:101E2000FC4F208349C080914C03282F30E03A8337
:101E3000298389819A81009731F029813A81213063
:101E4000310521F139C080912A04833271F48091E7
:101E50004D03882351F481E080934C03A5E3B0E067
:101E6000E5E3F0E0808188608C931092E403309188
:101E7000E403832F90E020912A04FC01E25BFC4FF5
:101E80002083832F8F5F8093E40316C08091E40347
:101E9000882F90E020912A04FC01E25BFC4F208314
:101EA0008091E403863930F48091E4038F5F80935E
:101EB000E40302C010924C030F900F90CF91DF917A
:101EC000FF91EF91BF91AF919F918F913F912F9192
:101ED0000F900FBE0F901F901895DF93CF93CDB743
:101EE000DEB76E970FB6F894DEBF0FBECDBF809100
:101EF000EA039091EB039E01255F3F4FB9014AE051
:101F000050E00E94D81080E4898384E48A8380E3CF
:101F10008B831C82CE010B960E94BF10AC019E01E8
:101F2000255F3F4FCE010196B9010E94C810CE0136
:101F300001960E94BF109C01CE010196820F931F53
:101F40002BE333E0B90142E050E00E94B610CE012D
:101F500001960E94490E8091EC039091ED039E0141
:101F6000255F3F4FB9014AE050E00E94D81080E45D
:101F7000898384E48A8381E38B831C82CE010B9660
:101F80000E94BF10AC019E01255F3F4FCE0101961C
:101F9000B9010E94C810CE0101960E94BF109C0199
:101FA000CE010196820F931F2BE333E0B90142E08B
:101FB00050E00E94B610CE0101960E94490E809119
:101FC000F4039091F5039E01255F3F4FB9014AE06C
:101FD00050E00E94D81080E4898388E68A838DE3EC
:101FE0008B831C82CE010B960E94BF10AC019E0118
:101FF000255F3F4FCE010196B9010E94C810CE0166
:1020000001960E94BF109C01CE010196820F931F82
:102010002BE333E0B90142E050E00E94B610CE015C
:1020200001960E94490E8091FC039091FD039E0150
:10203000255F3F4FB9014AE050E00E94D81080E48C
:10204000898386E58A838CE68B831C82CE010B967E
:102050000E94BF10AC019E01255F3F4FCE0101964B
:10206000B9010E94C810CE0101960E94BF109C01C8
:10207000CE010196820F931F2BE333E0B90142E0BA
:1020800050E00E94B610CE0101960E94490E809148
:102090004603909147039E01255F3F4FB9014AE0F7
:1020A00050E00E94D81080E4898386E58A8381E429
:1020B0008B831C82CE010B960E94BF10AC019E0147
:1020C000255F3F4FCE010196B9010E94C810CE0195
:1020D00001960E94BF109C01CE010196820F931FB2
:1020E0002BE333E0B90142E050E00E94B610CE018C
:1020F00001960E94490E6E960FB6F894DEBF0FBE91
:10210000CDBFCF91DF910895DF93CF93CDB7DEB7E9
:10211000A5E3B0E0E5E3F0E0908182E089278C93CD
:10212000CF91DF910895DF93CF93CDB7DEB7809144
:1021300045038130C1F480914403813051F4A5E31B
:10214000B0E0E5E3F0E080818E7F8C931092440351
:102150000AC0A5E3B0E0E5E3F0E0808181608C9304
:1021600081E080934403CF91DF910895FB01DC016E
:1021700002C001900D9241505040D8F70895FC01E3
:1021800001900020E9F7809590958E0F9F1F08958C
:10219000FB01DC010D900020E9F711974150504000
:1021A00028F0019000200D92C9F708951C9208951F
:1021B000FB019F01E8944230C4F04532B4F44A3048
:1021C00029F497FB1EF4909581959F4F642F7727F4
:1021D0000E941C11805D8A330CF0895D8193CB01D4
:1021E0000097A1F716F45DE251931082C9010C9497
:1021F000F910DC01FC01672F71917723E1F7329729
:1022000004C07C916D9370836291AE17BF07C8F3D1
:10221000089597FB092E07260AD077FD04D00CD02D
:1022200006D000201AF4709561957F4F0895F6F757
:10223000909581959F4F0895AA1BBB1B51E107C044
:10224000AA1FBB1FA617B70710F0A61BB70B881F46
:10225000991F5A95A9F780959095BC01CD010895D5
:04226000F894FFCF20
:1022640001125A2C294400000A310023002300548F
:1022740064665363655262005161005060005060AF
:102284000051610052620053636554646667686973
:102294006A6B6B6A696867555155554855552A15D7
:1022A40054AA8552AAA14008005548555548555589
:1022B4004855554855554855554855554855554020
:1022C40055555555555555555555555555555555BA
:1022D40055555555555555550000554AA85552A8BC
:1022E4005554A855522855484855215054855452A0
:1022F40015554855554155555555555555555555EB
:102304005555555555555555555555555555555579
:102314005555555555555555555555555555555569
:1023240055555555515555505555521555528500CD
:1023340002A12AAAA80002A155528555521555504A
:10234400555551555555555555555555555555553D
:102354005555555555555555555555555555555529
:10236400555555555555555555555555515555482A
:102374005555521555548554552150554848555274
:10238400285554A85552A8554AA8550000555555E6
:1023940055555555555555555555555555555555E9
:1023A4005555555540555548555548555548555515
:1023B400485555485555485555485540080052AA62
:1023C400A154AA85552A1555485555515555555565
:1023D40055555555555555555555555555555555A9
:1023E40055555555555555555555555555554555A9
:1023F40055215554851552150548552121552885D3
:10240400552A15552A85552AA15500005555555567
:102414005555555555555555555555555555555568
:102424005555555545555505555485555285554A67
:1024340080002AAAA84A800052855554855555051E
:102444005555455555555555555555555555555548
:10245400555555555555550000552AA1552A8555AC
:102464002A155528855521215505485515521555C8
:10247400548555552155554555555555555555551D
:1024840055555555555555555555555555555555F8
:0E24940055555555555555E8030D0A230000C2
:00000001FF
